:020000020000FC
:0200000057C0E7
:100080004A3220363530204D5352204669726D7702
:100090006172652056657273696F6E20312E332050
:1000A00020417072696C20312C20323030390000D0
:1000B00004E00EBF0FEF0DBF09E704B90FEF05B95C
:1000C00004E007B90AE308B900E20AB905E10BB98F
:1000D00080E090E087D4053561F105E573D40196A1
:1000E00001E070D48830D9F7019603E06BD4019613
:1000F0000FEF68D48C38D9F78DE601960CE762D4FF
:100100008337D9F701960FEF5DD48837D9F700E62A
:1001100059D401960FEF56D48238D9F781E8019669
:100120000CE750D48838D9F700E64CD484E60DE0CB
:1001300049D4A0E0B1E000E010E10D931A95E9F791
:10014000E894C2F800E0F02EC02E0093A7020FE959
:10015000602E85E042D4F02A12D417D40EE101D4E7
:100160000A95E9F741D13AEA57D2F0E0E0E8059183
:100170000A3461F40591023349F4FAE0E8E00591AC
:100180000E3421F405910F3609F402C010D4FECFCD
:100190009ED2D2D201D0FCCF4B9908950FD042D13C
:1001A0006DD189D1A6D10F2D087329F040D15ED130
:1001B000F2D31AD10895FBD317D108952E9A0000D7
:1001C00000002E9800004B99FECF00E110E020E0E7
:1001D0002E9A000000002E984B9B4B99111F221F56
:1001E0000A95A1F741E011D042E00FD044E00DD0D4
:1001F000F3FC0895F4FC0895F5FC089544E06DD0F7
:1002000042E06BD041E069D0089540FF07C0C8E2EA
:10021000D1E057E06FE370E285E20AC0CAE1D2E0C4
:1002200041FF02C0CDE8D1E055E06FE070E38BE321
:10023000A0E0B0E000E0E02E352F6894F6F8F7F883
:100240002E9A000000002E980000000088944B9B1E
:10025000089407953A9581F5573011F00695069563
:100260000695302F2227152F1A95369508F42395D9
:100270001A95D9F72170322759F00623D02E070F8F
:100280000993F7FA5EF4ED24F6FA1EF4081709F064
:1002900019C00F3369F4E894F7F80AC0ED1439F483
:1002A000689440FDF3F841FDF4F842FDF5F80AC00A
:1002B000E894F6F8352F00E00D90A03C12E0B1076D
:1002C00009F0BECF0D90A03C12E0B10729F02E9AA4
:1002D000000000002E98F6CF089540FF07C0C8E246
:1002E000D1E057E06FE370E285E20AC0CAE1D2E0F4
:1002F00041FF02C0CDE8D1E055E06FE070E38BE351
:10030000A0E0B0E000E0E02E352F6894F6F8F7F8B2
:100310002E9A000000002E98000000004B9B0CC09D
:100320000D90A03C12E0B10799F708952E9A0000B5
:1003300000002E980000000088944B9B08940795BD
:100340003A9589F5573011F0069506950695000007
:10035000302F2227152F1A95369508F423951A95D4
:10036000D9F72170322759F00623D02E070F0993B1
:10037000F7FA5EF4ED24F6FA1EF4081709F025C02A
:100380000F3369F4E894F7F80AC0ED1439F468946F
:1003900040FDF3F841FDF4F842FDF5F80895E894C6
:1003A000F6F8352F00E0A03C12E0B10709F40895FB
:1003B0000D90A03C12E0B10739F4F7FA26F006954B
:1003C0003A95E9F7BFCF0895B1CFA03C12E0B1074D
:1003D00051F00D90A03C12E0B10729F02E9A0000D8
:1003E00000002E98F2CF08952E9A00000000539A34
:1003F0007BD22E98000000002E9A000000002E985C
:100400000000539800002E9A000000002E98000073
:1004100000002E9A000000002E98E894F3F8F4F8FB
:10042000F5F808950F2D087391F08AE002C084E179
:1004300000C01AE0180FD1D20F3F49F08F931F93DD
:10044000802F76D01F918F9183958117A1F7089502
:100450008EE1EFCF88E2EDCF82E3EBCF8CE3E9CF03
:1004600086E4E7CF80E5E5CF8AE5E3CF84E6E1CF18
:100470008EE6DFCF88E7DDCF82E8DBCFF3FE08959D
:1004800086E0ABD200FF0895E3DF00E0402EC8E233
:10049000D1E08991F0FC04C08532D9F38F3319F093
:1004A00047D08F33B1F784E098D200FD02C0899124
:1004B0003FD0D0DF0895F4FE089587E08ED200FF8C
:1004C0000895D2DFC9DF00E0402ECDE8D1E0899168
:1004D000F0FC04C08B33D9F38F3319F029D08F335C
:1004E000B1F784E07AD200FD02C0899121D0B6DF55
:1004F0000895F5FE089588E070D200FF0895B4DFF6
:10050000AFDF00E0402ECAE1D2E08991F0FC04C0E8
:100510008B33D9F38F3319F00BD08F33B1F784E0DD
:100520005CD200FD02C0899103D09CDF9DDF08955D
:100530008032C0F08F3718F0FAE0EAEA67C0009125
:10054000A802047061F0813450F08B3530F08136B0
:1005500030F08B3724F400E2801B00E2800F17D0CC
:1005600040F120C08B3129F08D3051F010D0D8F1FE
:100570002DC036E751D030EF4FD036E74DD008953B
:100580003AE54AD030EF48D03AE546D00895FAE04F
:10059000EAE2082F10E0E00FF11FC895902D9F7739
:1005A000001C0895392F38D030EF36D0392F34D091
:1005B000089532E131D0392F2FD030EF2DD0392F9F
:1005C0002BD030EF29D032E127D0089534E124D068
:1005D000392F22D030EF20D0392F1ED030EF1CD051
:1005E00034E11AD0089532E117D034E115D0392F13
:1005F00013D030EF11D0392F0FD030EF0DD034E1C0
:100600000BD030EF09D032E107D008953591332374
:1006100011F002D0FBCF089573D13093AA027FD19D
:1006200047D1489B30C000E04A9905C0FDCF40D17A
:100630000A95D1F7F1CF632F112708E0669508F4EA
:1006400013950A95D9F761E0162732D1889412D014
:100650000894379501C03695771C303019F077949F
:1006600009D0F9CF179506D090D18CD121D187D15F
:100670001FD1089510F489D101C08AD183D118D136
:100680007ED116D108958894489908954A9BFECF4B
:100690000FD1332718E013D037951A95E1F70FD013
:1006A00071D106D16CD174D103D16CD101D16DD18E
:1006B00066D13F933AEFB4DF3F910894089562D139
:1006C000F7D08894489908945AD1F2D00895DBDF86
:1006D00008F008953F3F71F1323F11F13D3E29F19D
:1006E000333FC9F0353F79F03E3E19F0303F19F005
:1006F000089592DF0895C7DF303021F43AEF8CDFA0
:1007000030E08ADF0895BFDF343F00270093A9025D
:100710000093A8020895B7DF40F43093A90208952A
:100720003BEA7ADF33E878DF0895ADDFF0F7309306
:10073000A802089516D1BCCCC3D0389AC1D038983D
:1007400000D1309B0AC0BCD0C2FE03C033D0E894B5
:10075000C2F8E894C0F8C1F808956894C0F8C1FCE4
:100760000895AED02FD061F0ABD0389AA9D0389888
:10077000E8D0309BF2CFA4D0E894C0F8C1F8089537
:10078000C8E2D1E022E00A910F3F39F30F931F93A3
:100790002F936EDE2F911F910F913ED06894C1F878
:1007A000C2F80F931F932F9365DE2F911F910F9126
:1007B000F2D008950F931F932F935EDE2F911F9118
:1007C0000F910895C0E2D1E018E003E3389A92D087
:1007D000079508F43898B5D038988CD01A95B1F7A9
:1007E00028E018E0389A86D0389884D00894309B56
:1007F00088940795A6D01A95A9F70993283019F47B
:10080000013009F0089518E02A9561F73BD008956A
:10081000C7E2D1E026E003C0C8E2D1E028E00A91B7
:10082000069506950695069505D0088103D02A956C
:10083000B1F708950F700A301CF410E3010F02C0E5
:1008400017E3010F2F93802F73DE2F910895C0E2DD
:10085000D1E028E00881069506950695069505D015
:10086000099103D02A95B1F708950F700A301CF44E
:1008700010E3010F02C017E3010F2F93802F58DE02
:100880002F910895C0E2D1E028E030E018E009910E
:10089000402F432736950695469510F44CE83427AB
:1008A0001A95B1F72A9591F7C0E2D1E0303008955A
:1008B0000AE50A95F1F7089508E20A95F1F7089517
:1008C0000F930AE00BD00A95E9F70F9108950F9363
:1008D00005E004D00A95E9F70F9108950F9300E819
:1008E0000A95F1F70F9108950F930DE00A95F1F72E
:1008F0000F9108950F9302E00A95F1F70F91089573
:100900008F930F9389E069D0003019F405C0D8DFC8
:1009100003C005D00A95E9F70F918F9108950F93C1
:100920000FEF6AE06A95F1F70A95D9F70F910895EC
:100930000F930FEF66E16A95F1F70A95D9F70F91DA
:1009400008950F930AE0D0DF0A95E9F70F91089513
:100950000F9302E0EDDF0A95E9F7B2DFB1DF0F9107
:1009600008950F9305E0E4DF0A95E9F70F910895E4
:100970000F930EE1B9DF0A95E9F70F9108955298A8
:100980005A9A08955A98529A08955098589A0895E4
:100990005898509A089582E020D000FF089500E012
:1009A000429AE6DF4298E4DF0A95D1F7089581E0A4
:1009B00014D000FF0895F3DF0AE0D3DF0A95E9F7CA
:1009C000EEDF0895F999FECF0FB6F89492BD81BD80
:1009D00000BDFA9AF99A0FBE08959F9390E002D055
:1009E0009F910895F999FECF92BD81BDF89A00B507
:1009F0000895436F707972696768742028632920AD
:100A00003230303820432E204E6F726D616E20439D
:100A1000616D7062656C6C20616C6C2072696768D6
:100A2000742072657365727665649E1C322123247E
:100A30002B3433433B424B3A31444D152D1B2C3C58
:100A40002A1D22351A545D5BB6CE2996D2A6A5AED4
:100A5000BD52C6C5BED5414E494A45161E26252E55
:100A6000363D3E46CC4CC155C9CA9E9CB2A1A3A4FA
:100A7000ABB4B3C3BBC2CBBAB1C4CD95AD9BACBC18
:100A8000AA9DA2B59A545D5BB6CE0E1C32212324DA
:100A90002B3433433B424B3A31444D152D1B2C3CF8
:100AA0002A1D22351AD4DDDB8E00E071E0F07100E2
:00000001FF
